:020000040800F2
:1000000000040020E1010008A90D0008A90D000866
:10001000A90D0008A90D0008A90D0008A90D0008E8
:10002000A90D0008A90D0008A90D0008852F0008DA
:10003000A90D0008A90D0008A90D0008A90D0008C8
:10004000A90D0008A90D0008A90D0008A90D0008B8
:10005000A90D0008A90D0008A90D0008A90D0008A8
:10006000A90D0008A90D0008A90D0008A90D000898
:10007000A90D0008A90D0008A90D0008A90D000888
:10008000A90D0008A90D0008A90D0008A90D000878
:10009000A90D0008A90D0008A90D0008A90D000868
:1000A000A90D0008A90D0008A90D0008A90D000858
:1000B000A90D0008A90D0008A90D0008A90D000848
:1000C000A90D0008A90D0008A90D0008A90D000838
:1000D000A90D0008A90D0008892700089D27000820
:1000E000A90D0008A90D0008A90D0008A90D000818
:1000F000A90D0008A90D0008A90D0008A90D000808
:10010000A90D0008A90D0008E1250008A90D0008A7
:10011000A90D0008A90D0008A90D0008A90D0008E7
:10012000A90D0008A90D0008A90D0008A90D0008D7
:10013000A90D0008A90D0008A90D0008A90D0008C7
:10014000A90D0008A90D0008A90D000881230008C9
:10015000A90D0008A90D0008A90D0008A90D0008A7
:10016000A90D0008A90D0008A90D0008A90D000897
:10017000A90D0008A90D0008A90D0008A90D000887
:10018000A90D0008A90D0008B1270008A90D000855
:10019000A90D0008A90D0008A90D0008A90D000867
:1001A000A90D0008A90D0008A90D0008A90D000857
:1001B000A90D0008A90D0008A90D0008A90D000847
:1001C000A90D0008A90D0008A90D0008A90D000837
:1001D000A90D0008A90D0008A90D0008A90D000827
:1001E00072B6374880F3098836484EF60851CEF289
:1001F0000001086040F20000CCF200004EF63471BD
:10020000CEF200010860BFF34F8FBFF36F8F40F253
:100210000000C0F2F0004EF68851CEF200010860F6
:10022000BFF34F8FBFF36F8F4FF00000E1EE100A66
:100230004EF63C71CEF200010860062080F314886F
:10024000BFF36F8F00F092FD02F062FB4FF055306C
:100250001D491E4A91423CBF41F8040BFAE71C4974
:10026000174A91423CBF41F8040BFAE719491A4A70
:100270001A4B9A423EBF51F8040B42F8040BF8E7C0
:1002800000201749174A91423CBF41F8040BFAE796
:1002900000F070FD02F03EFB134C144DAC4203DA4B
:1002A00054F8041B8847F9E700F03EF8104C114D54
:1002B000AC4203DA54F8041B8847F9E700F058BD54
:1002C00000080020000000080000002000040020BA
:1002D00000040020483D00080008002028080020F5
:1002E0002808002090330020E0010008E001000809
:1002F000E0010008E00100082DE9F04F2DED108A23
:10030000C1F80CD0C3689D46BDEC108ABDE8F08FE3
:10031000002383F311882846A047002000F048FFFF
:1003200000F0E2FE00DFFEE770B51D4C092300255A
:1003300023706FF03F061F236570A570E57025716F
:100340006571A571E57125726672A372E57200F0A0
:100350002FFC20B10F2325726672A372E57202F0A2
:1003600033FD104B984217D00133984241F2883444
:1003700012BF002500240125002002F02BFD0DB145
:1003800000F054F800F098FC00F048FB204600F024
:1003900093F800F04BF8F9E700242546ECE700BF9E
:1003A00028080020010007B008B500F0B5FAA0F158
:1003B00020035842584108BD07B5054B02211B8850
:1003C000ADF8043001A800F013FB03B05DF804FBA6
:1003D0008C39000810B51148C3680BB100F0B0FDAE
:1003E0000F4C104A0D4800234FF47A7100F06CFD59
:1003F000236813B12368013B2360636813B163680A
:10040000013B6360084B1B7833B9636823B9022052
:1004100000F00CFC3223636010BD00BF34080020E4
:100420004C0D0020D50300084808002038B51B4CAF
:100430002368013330D01A4D1A4B2A689A422BD9BF
:10044000194B9B6803F1006303F580439A4223D262
:10045000002000F0FDFA154B0220187000F0DCFBC4
:10046000134B1A6C00221A64596C5A64596941F092
:10047000800159615A61196941F0005119611A618D
:1004800072B60C4B1C6023682A68202181F3118806
:100490009D4683F30888104738BD00BF0040000820
:1004A00004400008FF3F00082808002048080020FA
:1004B0000038024008ED00E02DE9F04FB34B8246D2
:1004C000B3489C680022C2608FB0202282F311885A
:1004D000C26800930AB100F033FD0023AD4AAC4876
:1004E0004FF47A7100F0F0FC002383F31188DFF8F9
:1004F000C0B2BAF1000F01D0CBF800A0A64FCBF8E4
:10050000043000253B702E464FF0FF38012000F0EC
:1005100083FBBAF1000F00F0C181DBF80030002B43
:1005200040F0BC810FB0BDE8F08F0220FFF73CFF28
:10053000002840F0AF81994B1B88ADF82430022190
:1005400009A800F055FAE1E74FF47A7000F0E4F9F9
:10055000031E0193EFDB0220FFF726FF81460028F0
:10056000E9D0019B581E0428E5D8DFE800F003100D
:10057000131619000EA8052340F8143D042100F0BD
:1005800037FA4D4600F08EFBFFF716FF7FE104219E
:100590007E48F4E704218248F1E704218148EEE730
:1005A0001C25284600F056FA04350990042109A8B4
:1005B00000F01EFA2C2DF4D1E3E7002EBBD0002D65
:1005C000B9D00220FFF7F0FE064610B901252E46ED
:1005D000B1E7012000F03CFA0220387000F01CFB6B
:1005E00000255FFA85F9484600F04AFA01350446CD
:1005F00018B1484600F054FAF3E7012302203B709B
:1006000000F000FB009B9B689C4207D2204600F054
:1006100021FA013040F040810434F3E700243C70BB
:10062000CBF804403546ADE7002E84D0002D82D0B3
:100630000220387000F0F0FA322000F06DF9051E4B
:10064000C4DB15F00306C1D1009A92686319934286
:10065000BCD8B5F5807FB9D8DFF84C91AE420CDA42
:100660004FF47A7000F058F90390039B002BADDB38
:10067000039B06F809300136F0E7C820FFF794FE27
:1006800006460028A2D02CB9474B4FF0FF32D3F8D2
:1006900000801A60444B25F003052544A3EB0409B0
:1006A000AC42BFD059F80410204600F0D9F92046DA
:1006B00000F0D0F959F80430984240F0ED8004344D
:1006C000EEE70220FFF770FE00283FF434AF4FF052
:1006D000000AD146009B9B689A4537D2BAF1000FB9
:1006E00017D1B8F1FF3F14D0CDF824802F494B68C3
:1006F000A3B1002209A8135C83EA0903DBB201322B
:1007000051F82330042A83EA1929F4D10AF1040AA2
:10071000E0E7504600F09EF90990E7E71A46082006
:1007200012F0010F4FEA52021FBF82F06D4282F4B5
:10073000380282F4034282F020020138F0D141F8FD
:1007400023200133B3F5807FE8D1D2E70EA804213E
:1007500040F8289D00F04CF914E70EA8002340F85B
:10076000143D642100F010F900287FF4E4AE02206B
:10077000FFF71AFE00283FF4DEAE099800F0A2F958
:100780000EAB43F8240D04211846E3E728080020A7
:1007900034080020D5030008480800208E390008DE
:1007A0002C080020300800204C0800204C090020B4
:1007B0004C0D00200EA8002340F8143D642100F0E9
:1007C000E3F800287FF4B7AE0220FFF7EDFD002824
:1007D0003FF4B1AE099800F083F90EAB43F8200D59
:1007E000D1E70220FFF7E0FD00283FF4A4AE00F0BF
:1007F0007DF90EAB43F81C0DC5E70220FFF7D4FDD1
:1008000000283FF498AE09A9142000F075F981463C
:100810000EA8042140F8189D00F0EAF8494609A8FE
:1008200098E74FF47A70FFF7BFFD00283FF483AEDE
:10083000B8F1FF3F05D1FFF7BFFD354800F0BEFC22
:1008400070E64146002000F00BF9002000F002F9AC
:100850008045F0D02F4B6FE60EA8002340F8143DE2
:10086000642100F091F800287FF465AE0220FFF7C4
:100870009BFD00283FF45FAEFFF79EFD41F28830FC
:1008800000F09CFC099800F051FA00F00BFA4FF0D0
:10089000000A3BE6064675E63546DBE7002000F039
:1008A0003BF80390039B002BFFF633AE012000F0D2
:1008B000A9F9039B213B122B3FF628AE01A252F867
:1008C00023F000BF2B05000849050008BB05000800
:1008D0000D0500080D0500080D0500082906000893
:1008E0000D050008C30600085B070008B5070008EF
:1008F000E30700080D050008FB0700080D050008C8
:1009000023080008850500080D050008590800089F
:10091000A0860100903900082DE9F34702AE0024BB
:100920004FF47A7506F8014D144FDFF858804543AF
:1009300097F900305A1C5FFA84F901D0A34212D112
:1009400058F8240003680122D3F81CA031462B4636
:10095000D047012807D10A4B9DF8070083F8009083
:1009600002B0BDE8F0870134042CE1D14FF4FA70F5
:1009700000F024FC4FF0FF30F2E700BF0008002039
:100980006C0D0020E43900082DE9F0474FF47A752A
:10099000144FDFF8588006464D43002497F9003085
:1009A0005A1C5FFA84F901D0A34210D158F82400F0
:1009B00003680422D3F81CA031462B46D0470428F4
:1009C00005D1094B83F800900020BDE8F087013481
:1009D000042CE3D14FF4FA7000F0F0FB4FF0FF303D
:1009E000BDE8F087000800206C0D0020E439000805
:1009F00030B4074B1A78074B53F8224023689D699F
:100A0000054B0A46AC460146204630BC604700BF55
:100A10006C0D0020E4390008A086010070B502F0DA
:100A200009F9094C094E207000253068237883426B
:100A300008D902F0F9F8336805440133B5F5804F61
:100A40003360F2D370BD00BF6D0D0020540D002047
:100A500002F0A6B900F1006000F580400068704720
:100A600007B502AB00F1006043F8041D04221946EB
:100A700000F5804002F022F903B05DF804FB0000AD
:100A8000054B1A68054B1B781344834202D9104466
:100A900002F0CAB800207047540D00206D0D0020F0
:100AA00038B5074D04462868204402F0C5F828B937
:100AB00028682044BDE8384002F0D6B838BD00BFF1
:100AC000540D002010F0030308D1B0F5007F05D8C5
:100AD00000F10050A0F50840006870470020704702
:100AE000014BC058704700BF107AFF1F014B1868B8
:100AF000704700BF002004E070B52A4B1C68C4F3A7
:100B00000B03240C63B140F21342934231D040F204
:100B1000194293422FD040F2214293422DD1032318
:100B2000214A0C2505FB03235D6893F9082042F256
:100B300001039C4224D0B4F5805F23D041F201032D
:100B40009C4221D041F203039C421FD041F2070393
:100B50009C4208BF3122441E0C44013D0B46A34277
:100B60001ED215F9016F581C96B1034600F8016CAE
:100B7000F5E70123D4E70223D2E73F220B4DD6E766
:100B80003322E3E74122E1E75A22E4E75922E2E790
:100B90002C2584421D7001D9981C5A70401A70BDD2
:100BA0001846FBE7002004E0B43900089439000837
:100BB000124B5A8842F201018A4293B214D0B3F523
:100BC000805F13D041F20102934211D041F203023F
:100BD00093420FD041F2070293420DD10423084AF9
:100BE00002EB8303D87870470023F8E70123F6E788
:100BF0000223F4E70323F2E700207047002004E01B
:100C0000A0390008022802BF024B4FF480529A61BB
:100C1000704700BF00100240022802BF024B4FF095
:100C200080529A61704700BF00100240022801BF45
:100C3000024A536983F480535361704700100240A5
:100C400010B50023934203D0CC5CC4540133F9E7C0
:100C500010BD000030B5441E14F9010F0B4660B101
:100C600093F90050854201F1010106D11AB993F9B7
:100C70000020801A30BD013AEEE7002AF7D1104675
:100C800030BD000002460346981A13F9011B0029E3
:100C9000FAD1704702440346934202D003F8011B85
:100CA000FAE77047024B1A78024B1A70704700BF80
:100CB0006C0D002000080020F8B5164C1648174DA2
:100CC000174E154F00F0AEFB2146134800F0D6FB3F
:100CD000236814485A6D936B23F40023936300F048
:100CE0006DFA2068104900F0E5FC23685A6D936B9B
:100CF00043F4002393634FF4E1332B60002456F850
:100D00002400B84202D0294600F0F2FA0134042C43
:100D1000F5D1F8BDF43B0008082A0020580D00204A
:100D2000E439000840420F00443C000838B50B4B42
:100D30001A780B4B53F822400A4B9C4205460CD0C4
:100D4000094B002118461422FFF7A4FF0560014655
:100D50002046BDE8384000F0CBBA38BD6C0D00200D
:100D6000E4390008082A0020580D002070470000D0
:100D7000FEE70000084A094B09498B4204D3094A9F
:100D80000021934205D3704752F8040F43F8040B37
:100D9000F3E743F8041BF4E76C3D000890330020B0
:100DA00090330020903300201EF0040F0CBFEFF3AF
:100DB0000880EFF309808169004A1047C50D0008DB
:100DC00070470000204B02681A60204B42681A608E
:100DD0001F4B82681A601F4BC2681A601E4B026963
:100DE0001A601E4B42691A601D4B82691A601D4BC6
:100DF000C2691A601C4B1D491A681D4B1A601A689B
:100E0000120A0A701A681B4B1A701B4B1A681B4B8C
:100E10001A601B4B1A681B4B1A601B4B1A681B4B42
:100E20001A601B4B1A681B4B1A601B4B1A681B4B32
:100E30001A601B4B5A6A1B4B1A601B4B1B68DB0763
:100E400001D500BEFEE7FEE7A00D0020A40D0020A6
:100E5000AC0D0020B00D0020A80D0020940D002046
:100E6000980D00209C0D002028ED00E0780D00205A
:100E70007C0D00208C0D00202CED00E0840D002066
:100E800030ED00E0800D00203CED00E0700D002012
:100E900034ED00E0880D002038ED00E0740D0020F6
:100EA00000ED00E0900D0020F0ED00E0054B03F1B7
:100EB00014025A619A614FF0FF32DA6100221A621D
:100EC000704700BFB40D0020F8B503611A4BC26033
:100ED0005C6A1A4B1A46022952F8145F38BF022185
:100EE000954206461F460AD1586198611C6205600A
:100EF000456081600819BDE8F84000F0B5BB186A8C
:100F0000AB68241A0C1902D3E41A2D6804E09C4241
:100F100002D2204400F0B8FBAB689C42F4D86B6866
:100F2000736035601E606E60B460A9684FF0FF3377
:100F3000091BA960FB61F8BD000C0040B40D002046
:100F400010B41A4C234653F8141F814210D0416844
:100F500002680A60026851609A424FF00001C16065
:100F600003D0936881680B4493605DF8044B70472D
:100F70000A68626100209A425360C86003D15DF83C
:100F8000044B00F07BBB9368886803449360084A75
:100F9000506A226A821A9342E7D99B1A022B2CBF0D
:100FA000C01802305DF8044B00F06EBBB40D002099
:100FB000000C0040024B00221B605B609A6070478F
:100FC000B40D0020002303748268054B1B689968E8
:100FD0009142FBD25A6803604260106058607047CB
:100FE000B40D002008B5202383F31188037C032B64
:100FF00005D0042B0DD02BB983F3118808BD4369AC
:1010000000221A604FF0FF334361FFF7DBFF00233C
:10101000F2E790E80C001A6002685360F2E7000003
:10102000002303748268054B1B6899689142FBD8C2
:101030005A6803604260106058607047B40D002029
:10104000054B19690874186802681A6053601861C2
:1010500001230374FFF750B9B40D002030B54B1CC9
:1010600087B005460A4C10D023690A4A01A8FFF749
:101070002BFF2846FFF7E4FF049B13B101A8FFF7FD
:101080005FFF2369586907B030BDFFF7D9FFF8E764
:10109000B40D0020E50F000838B50C4D41612B69F7
:1010A00081689A689142044603D8BDE83840FFF74A
:1010B00089BF1846FFF786FF01232C610146237480
:1010C0002046BDE83840FFF717B900BFB40D002037
:1010D000044B1A681B6990689B68984294BF002073
:1010E00001207047B40D002010B5084C236820691A
:1010F0001A6822605460012223611A74FFF790FF7E
:1011000001462069BDE81040FFF7F6B8B40D002095
:1011100008B5FFF7DDFF18B1BDE80840FFF7E4BFF1
:1011200008BD0000826002220274002242748261C3
:10113000704700008368A3F1840243F8142C02690D
:1011400043F8442C426943F8402C084A43F8242CC5
:10115000C26843F8182C022203F8102C002203F86E
:101160000F2C43F8082CA3F120007047110300084E
:1011700008B5FFF7DFFFBDE80840FFF723BF000019
:1011800010B5202383F31188FFF7D4FF0021044614
:10119000FFF782FF002383F31188204610BD000073
:1011A000024B1B6958610F20FFF74ABFB40D0020A6
:1011B000202383F31188FFF7F3BF000008B5014631
:1011C000202383F311880820FFF748FF002383F3CF
:1011D000118808BD10B5054C2369036058610320D0
:1011E000FFF72EFF2369586910BD00BFB40D002022
:1011F00003682BB10022026059611846FFF7E2BE76
:101200007047000049B1064B42681B6918605A607C
:10121000136043600420FFF721BF4FF0FF30704799
:10122000B40D00200368984206D01A68026050602E
:1012300059611846FFF7C6BE7047000038B504462E
:101240000D462068844200D138BD036823605C608D
:101250004561FFF7B7FEF4E70C3002F02FB900004C
:101260004FF0FF330C3002F029B90000303002F0AB
:10127000C5B900004FF0FF33303002F0BFB90000B5
:101280000C3002F0F5B800004FF0FF310C3002F0E6
:10129000EFB80000303002F06FB900004FF0FF32BD
:1012A000303002F069B9000001F08CBA37B503465E
:1012B00015460E4A43F8042B43600123044603728B
:1012C0004FF4806200900B4600F154010C3002F0A4
:1012D000A5F800942B464FF4806204F2544104F1C7
:1012E000300002F03DF903B030BD00BF143A0008F1
:1012F00010B52023044683F3118801F093FA0223EA
:101300002372002383F3118810BD000038B54369B0
:1013100004460D461BB90421084401F00FFE29467E
:1013200004F10C0002F088F8002806DA201D4FF4C2
:101330008061BDE8384001F001BE38BD13B5446B93
:10134000D4F88C341A681178042916D1217A02292C
:1013500013D11979128901238B4013420DD101A9B0
:1013600004F1440001F06EFF024630B1D4F88C4421
:10137000019B2179206800F0E9F902B010BD00005E
:101380000C3001F0DBBE00004FF0FF330C3001F0F9
:10139000D5BE0000443001F0C1BF00004FF0FF3364
:1013A000443001F0BBBF00000C3001F0A9BE0000CA
:1013B0004FF0FF310C3001F0A3BE0000443001F0CB
:1013C0008DBF00004FF0FF32443001F087BF0000B6
:1013D000D0F88C2438B5136819780429054601D053
:1013E000012038BD017A0229FAD112795C890120E5
:1013F00090400440F4D105F10C0001F03BFE0246A0
:101400000028EDD0D5F88C544FF4807328686979A2
:1014100000F08AF9204638BD406BFFF7D9BF0000C5
:10142000704700007FB50346114A43F8042B01259D
:10143000436002260F4B057204460290019300F1AF
:101440007C02294600964FF480730C3001F0EEFDCB
:10145000094B0193029400964FF4807304F52172B6
:10146000294604F1440001F0C9FE04B070BD00BF7C
:10147000343A0008191400083D1300080B682022B4
:1014800082F311880A7903EB820290614A7909326A
:1014900043F822008A7912B103EB82039861022398
:1014A0000372C0F88C14002383F311887047000086
:1014B00038B5044601250221043001F03FFD04F156
:1014C0000C0025756FF00101FFF7B8FE84F84C5051
:1014D00004F144006FF00101BDE83840FFF7AEBEF3
:1014E00010B501210446043001F028FD00232375C6
:1014F00084F84C3010BD000038B5044600250C308F
:1015000001F0ACFD04F14400257501F08FFE201DB3
:1015100084F84C50012101F011FD2046BDE838400F
:10152000FFF756BF90F8443003F06003202B19D129
:1015300090F84520212A0AD0222A4FF000030ED02D
:10154000202A0FD1084A82630722C26304E0064BB7
:1015500083630723C363002303640120704783630D
:10156000C363F9E70020704701080020D0F88C34ED
:1015700037B51A681178042904461AD1017A02296C
:1015800017D11979128901238B40134211D100F12F
:101590004405284601F022FF58B101A9284601F070
:1015A00051FED4F88C44019B21790246206800F05A
:1015B000CDF803B030BD000000EB8103F7B59C69A6
:1015C00005460E46F4B1202383F3118805EB860708
:1015D000201D082101F0B2FCFB685B691B684434E4
:1015E00013B1204601F03CFE01A9204601F02AFE7D
:1015F000024648B1019B3146284600F0A7F8002377
:1016000083F3118803B0F0BDFB685A691268002AA1
:10161000F5D01B8A013B1340F1D105F14402EAE702
:10162000093110B550F82140CCB1202383F3118843
:101630000421601801F082FCD4F88C2413685279DC
:1016400003EB820304F10C00DB689B69596801F02D
:101650001BFD2046FFF7BCFE002383F3118810BD5D
:101660007047000000F0D0BF034B002258631A619E
:101670000222DA60704700BF000C0040014B0022DC
:10168000DA607047000C0040014B5863704700BFA0
:10169000000C004000F09CBB01230370002343605A
:1016A000C36183620362C362436203630381438154
:1016B0007047000038B50446202383F311880025C5
:1016C0004160C56005614561856100F093FB0223BF
:1016D000237085F3118838BD70B500EB8103054692
:1016E0005069DA600E46144618B110220021FFF747
:1016F000D1FAA06918B110220021FFF7CBFA3146C8
:101700002846BDE8704000F04DBC0000028902F0A0
:1017100001020281428902F001024281002202613B
:101720004261826100F0D2BCF0B400EB81044789D1
:10173000E4680125A4698D403D4345812360002371
:10174000A2606360F0BC00F0EDBC0000F0B400EB00
:1017500081040789E468012564698D403D43058162
:1017600023600023A2606360F0BC00F06BBD00004A
:1017700070B50223002504460370A0F84C5080F891
:101780004E5080F84F5005814581C5600561456127
:10179000856180F8345000F0A3FB63681B6823B1B7
:1017A00029462046BDE87040184770BD436802785E
:1017B0001B6880F85020052202700BB104211847E5
:1017C00070470000436890F850201B6802700BB10E
:1017D000052118477047000070B50023044680F8C3
:1017E000343000F1440200F093FC63689B685BBBFB
:1017F00094F8445015F0600614D194F8453005F083
:101800007F0545EA0325B5F5407F00F0A58059D84E
:10181000022D00F0F1803FD8002D00F08780012DCF
:1018200000F0E4800021204600F0BCFE00212046AC
:1018300000F0AEFE63681B6813B10621204698478E
:10184000062384F8343070BD204698470028CFD056
:1018500094F84B2094F84A3043EA0223E26B934217
:1018600038BFE36394F94430E56B002B4FF020035D
:1018700080F20181002D00F0F080012284F83420F4
:1018800083F311880021E36BA26B2046FFF75EFF14
:10189000002383F3118870BDB5F5807F4DD0B5F579
:1018A000817FBFD194F84630002BBBD194F84830EB
:1018B00013F00F0126D01A06204640F1B78000F041
:1018C00085FE1FE0B5F5C06F50D020D840F202333E
:1018D0009D4200F0AE80B5F5A06FA3D1B4F84430BE
:1018E000B3F5A06F0ED194F8463084F84E30204600
:1018F00000F04CFB63681B6813B101212046984738
:10190000032323700023A363E3632364A0E7B5F5F7
:10191000106F41D040F602439D4267D0B5F5006F8D
:1019200080D104F14F03A363012333E004F14C039E
:10193000A3630223E36325648AE794F84630012B0E
:101940007FF470AFB4F84C3023F00203A4F84C30AD
:10195000A663E66326647BE794F84630012B7FF4A8
:1019600061AFB4F84C3043F00203EFE794F849203C
:10197000616894F848304D6894F8471043EA0223B0
:10198000204694F84620A84700283FF44BAF436810
:10199000A3630368E363DDE794F84F2094F84630CF
:1019A0009A42AFD02378042B10D1202383F31188DF
:1019B0002046FFF7ABFE86F31188636884F84F601A
:1019C0001B68032121700BB12046984794F84630DC
:1019D000002B97D084F84F300423237063681B6872
:1019E000002B8FD00221204698478BE72E4BA36314
:1019F0000223E363002388E794F8481011F0800F76
:101A0000204601F00F010ED000F074FB012806D033
:101A100002287FF407AF254BA363E0639AE7244BCA
:101A2000A363E56396E700F057FBEFE700F0C4FD22
:101A300068E794F84630002B7FF4F4AE94F8483011
:101A400013F00F013FF45EAF1B06204602D500F0F5
:101A5000A9FD57E700F09CFD54E7032284F83420E9
:101A600083F311882B462A4629462046FFF75CFE61
:101A700085F3118870BD5DB1042284F8342083F3AE
:101A800011880021E36BA26B2046FFF74DFEFFE6B5
:101A9000052284F8342083F311882B462A462946F0
:101AA0002046FFF753FEE3E75C3A0008543A00088B
:101AB000583A000838B590F834300446062B22D83E
:101AC000DFE803F0370422373732370090F84B1045
:101AD00090F84A20C36B42EA01229A4214D9C268A4
:101AE000128AB3FBF2F502FB15356DB9202383F39F
:101AF00011882B462A462946FFF728FE85F31188D0
:101B0000022384F8343038BD032384F83430202392
:101B100083F3118800231A4619462046FFF704FE76
:101B2000002383F3118838BD036C03B19847002369
:101B3000E7E7002100F036FD0021204600F028FDF7
:101B400063681B6813B10621204698470623D8E72F
:101B500090F83420062A38B5044621D80123934052
:101B600013F0670F1DD113F008050FD1DB0617D551
:101B7000052380F83430202383F311882B462A462E
:101B80002946FFF7E3FD85F3118838BDC3689B69DB
:101B90005B682BB9036C03B19847002384F8343099
:101BA00038BD002100F0FEFC0021204600F0F0FCD2
:101BB00063681B6813B10621204698470623EDE7AA
:101BC000836D30B500229D68446D11464FF0FF30A3
:101BD00004EB421301329542C3F80019C3F81019FF
:101BE000C3F80809C3F8001BC3F8101BC3F8080B9F
:101BF000EED24FF00113C4F81C3830BD890141F01A
:101C00002001016103699B06FCD4122001F078B920
:101C10002DE9F04F202387B00446456D83F31188EA
:101C200000F1640305934FF0000B2378012B04D0DF
:101C3000236E4BB96B69DB0606D4AB69059843F09C
:101C40001003AB61FFF7C6FA8BF311884FF0000E5B
:101C50004FF02009A36D9B685FFA8EF083421BD280
:101C6000202383F31188E0E7616D0A6A02F4F01320
:101C7000B3F5802F66D0B3F5402F0DD1C2F30A160D
:101C800002F00F0204EB820201F58051D3681F6A53
:101C900000231A469E4248D1696911F01001E3D130
:101CA000012303FA00F2236E1A4200F08C8089F3BC
:101CB0001188AB6823F00103AB60236E23EA0203B3
:101CC000236681F3118804EB8003D3F80C80D8F8E5
:101CD00014100B680093431C1B03029343010493ED
:101CE0004868009B98425FD2B8F81060676D1B1A75
:101CF000B34228BF3346049EBE19D6F81869B6B25F
:101D0000B3EB860F62D8029EBE1903968E680196C9
:101D1000A6F1040A9C46039E5AF8047F3760BCF182
:101D2000040F3BD9ACF1040CF5E713F0030F08BF27
:101D30000A68072B98BF3A7003F101039CBF120A8F
:101D40000137A7E7C2F30A1602F00F0204EB820282
:101D500001F58051D3689B691F68D3F808805B68E0
:101D6000A7EB030C00231F469E4208D1D368996954
:101D70008A684B68324433448A604B608CE713F0C6
:101D8000030F08BF0F689C4588BF88F8007003F1F7
:101D9000010384BF3F0A08F10108E5E7019E1E44E4
:101DA00003448E604B609BE7012189F31188AB6887
:101DB00043F00103AB6021B9D5F834381A43C5F8B4
:101DC00034288BF311880EF1010E43E70021ECE774
:101DD00010B5064C2046FFF75FFC4FF0A0420023F1
:101DE0006265034A6366A265A36610BDF80D002014
:101DF000843A000870B50378012B86B005465BD1A4
:101E00002F4B446D984213D12E4B5A6B42F08002F7
:101E10005A635A6942F080025A6100225A610E21C7
:101E2000432001F03DFC284BE360284BC4F8003808
:101E300000232B66C4F8003EC02323604FF45023D8
:101E4000A3636E6D202001F05BF8012333613369D9
:101E5000DB07FCD4122001F053F83369002BFCDAC5
:101E60000026A6602846FFF7ABFE6B68C4F8106832
:101E7000DB68C4F81468C4F81C68FBB9144BA36190
:101E80004FF0FF336361AB6E93B9124B009305F1D2
:101E90007003019305F5367302930223039368469A
:101EA0000D4B04930595FFF763F9A866FFF730F92A
:101EB000A36843F00103A36006B070BD074BDEE7E3
:101EC000F80D0020003802404014004003002002BA
:101ED000003C30C0903A0008111C0008083C30C09B
:101EE000F8B5446D054600212046FFF787FEA96D31
:101EF00000234FF001128F68C4F834384FF00066A9
:101F0000C4F81C284FF0FF3004EB431201339F420A
:101F1000C2F80069C2F8006BC2F80809C2F8080BE1
:101F2000F2D20B68EB6563626B6D10221A611E6959
:101F300016F01006FBD1122000F0E2FFD4F80038B2
:101F400023F4FE63C4F80038A36943F4402343F04C
:101F50001003A3610923C4F81038C4F81438094BDE
:101F6000EB60094BC4F8106BC4F8003BC4F810696F
:101F7000C4F80039EB6D03F1100243F48013EA65F5
:101F8000A362F8BD603A000840800010426D90F8EE
:101F90004E10D2F8003823F4FE6343EA0113C2F86E
:101FA000003870472DE9F0410EB200EB86080D466F
:101FB000D8F80C100F6807F00303022B50D0032B46
:101FC00050D03D4A3D4F012B18BF1746446D4FEA94
:101FD000451E04EB0E030022C3F8102B8A6905F19D
:101FE000100C002A40D04A8A05F158035B013A439D
:101FF000E2500123D4F81C2803FA0CF31343A6443F
:102000004A69C4F81C380023CEF8103905F13F03A3
:10201000002A39D00A8A898B9208012988BF4A434D
:10202000C16D04EB8303561841EA0242C665294696
:102030005A602046FFF7E2FDD8F80C301B8A43EACD
:1020400085531F4305F148035B01E7500123D4F892
:102050001C2803FA05F51543C4F81C58BDE8F081A7
:10206000174FB3E7174FB1E704EB4613D3F8002B34
:1020700022F40042C3F8002BD4F81C28012303FAF1
:102080000CF322EA0303BAE704EB83030E4A5A6017
:1020900004EB461629462046FFF7B0FDD6F8003976
:1020A00023F40043C6F80039D4F81C38012202FAA0
:1020B00005F523EA0505CFE7008000100080041035
:1020C0000080081000800C1000040002826D12686D
:1020D000C265FFF775BD00005831436D49015B587B
:1020E00013F4004004D013F4001F14BF0120022099
:1020F000704700004831436D49015B5813F40040BC
:1021000004D013F4001F14BF012002207047000008
:1021100000EB8101CB68196A0B6813604B68536050
:102120007047000000EB810330B5DD68AA691368D1
:10213000D36019B9402B84BF402313606B8A1468A5
:10214000426D1C44013CB4FBF3F46343033323F0BE
:10215000030302EB411043EAC44343F0C043C0F819
:10216000103B2B6803F00303012B09B20ED1D2F808
:10217000083802EB411013F4807FD0F8003B14BF05
:1021800043F0805343F00053C0F8003B02EB411290
:10219000D2F8003B43F00443C2F8003B30BD0000DE
:1021A0002DE9F041264D6E6D06EB40130446D3F841
:1021B000087BC3F8087B38070AD5D6F81438190706
:1021C00006D505EB84032146DB6828465B68984703
:1021D000FA0733D5D6F81438DB072FD514B995F89C
:1021E00034305BB305EB8403D968CCB98B69488A7A
:1021F0005E68B6FBF0F200FB12628AB91868DA6812
:1022000090420DD2121A83E81400202383F3118820
:102210000B482146FFF786FF84F31188BDE8F08163
:10222000012303FA04F26B8923EA02036B81CB6872
:1022300023B121460248BDE8F0411847BDE8F081CE
:10224000F80D002000EB810370B5DD68436D6C690B
:102250002668E6604A0156BB1A444FF40020C2F8D3
:1022600010092A6802F00302012A0AB20ED1D3F83B
:10227000080803EB421410F4807FD4F8000914BF5F
:1022800040F0805040F00050C4F8000903EB4212C7
:10229000D2F8000940F00440C2F80009D3F834082D
:1022A000012202FA01F10143C3F8341870BD19B9D3
:1022B000402E84BF4020206020682E8A841940F080
:1022C0000050013C1A44B4FBF6F440EAC440C6E7AF
:1022D0002DE9F041284C666D06EB40130546D3F816
:1022E0000879C3F80879F9071AD5D6F81038DA074B
:1022F00016D504EB8003D9684B691868DA689042F8
:102300002CD2121A4FF000081A60C3F80480202360
:1023100083F3118829462046FFF794FF88F311883C
:102320003B0619D5D6F83428012303FA05F51542E2
:1023300012D0202383F31188236E10482B43236689
:10234000D6F8343823EA0505C6F834580021FEF7DC
:102350004FFF002383F31188BDE8F081012303FAC6
:1023600005F2238923EA020323818B68002BD7D04F
:10237000294620469847D3E7F80D00205C0E002040
:102380002DE9F74F8048446D6669A3691E4016F435
:10239000805F6661054608D000230366FFF7E8F911
:1023A00003B0BDE8F04F00F0FFBD002E12DAD4F804
:1023B000003E75489F071EBFD4F8003E23F003037C
:1023C000C4F8003ED4F8043843F00103C4F80438DC
:1023D000FFF7F8F9300504D500236B482B66FFF7AB
:1023E000E5F9B1040CD5D4F8083813F0060FE3680A
:1023F00023F470530CBF43F4105343F4A053E36031
:10240000320704D56B68DB680BB15F489847F3026D
:102410004ED4B7020CD5D5F85480DFF86CA1002754
:102420004FF00109AB6D9B68F9B28B4280F08F8051
:10243000F5060DD5202383F31188A369534823F0B3
:102440001003A3610021FEF7D3FE002383F311885C
:102450003003D4F8184813D5E10302D50020FFF764
:102460009FFEA20302D50120FFF79AFE630302D567
:102470000220FFF795FE270302D50320FFF790FE09
:1024800075038DD5E00702D50020FFF721FFA107D6
:1024900002D50120FFF71CFF620702D50220FFF7DB
:1024A00017FF23077FF57CAF0320FFF711FF77E7C6
:1024B000D5F854A0DFF8D4B04FF00009AB6D9B689D
:1024C0005FFA89F7BB42A4D30AEB4713D3F800297C
:1024D00002F44022B2F5802F36D1D3F80029002A29
:1024E00032DAD3F8002942F09042C3F80029D3F839
:1024F0000029002AFBDB3946686DFFF77FFB0123CB
:102500002A89BB406FEA030808EA02022A8105EB28
:102510008702D268926822B139461B4801939047DE
:10252000019B202282F31188DAF8342808EA02029B
:10253000CAF834282A6E0021134358462B66FEF74A
:1025400057FE002383F3118809F10109B6E708EB70
:102550004112D2F8003B03F44023B3F5802F10D191
:10256000D2F8003B002B0CDA6A8909FA01F322EA5F
:1025700003036B8105EB8103DB68DB680BB150461D
:10258000984701374EE700BFF80D00205C0E002091
:10259000436D03EB4111D1F8003B43F40013C1F844
:1025A000003B7047436D03EB4111D1F8003943F410
:1025B0000013C1F800397047436D03EB4111D1F8A6
:1025C000003B23F40013C1F8003B7047436D03EB5D
:1025D0004111D1F8003923F40013C1F800397047D4
:1025E000084B1A69920710B508D500241C612023F6
:1025F00083F3118800F04AFC84F31188BDE8104091
:1026000000F0D2BC000C00400D4A136C43F00803EC
:1026100013640C4A936843F0080393600A4B5322F7
:102620009A624FF0FF32DA6200229A615A63DA60EE
:102630005A6001225A6108211A60322001F030B834
:1026400000380240002004E0000C0040024AD36839
:1026500043F08003D360704700440040024AD368CF
:1026600043F08003D360704700480040024AD368BB
:1026700043F08003D3607047007800402DE9F041BB
:10268000D0F85468F7683368DA0505469CB20DD572
:10269000202383F311884FF40071043000F04EFCC6
:1026A0006FF480733360002383F31188202383F356
:1026B000118805F1040814F02F033AD183F311882F
:1026C000390617D5220615D5202383F3118805F185
:1026D000300000F079FF00284DDA0821281D00F0B5
:1026E0002DFC4FF63F733B4043F04003F360002363
:1026F00083F31188630614D5202383F311886A6C51
:10270000AB6C9A4202D1AB6B002B36D127F040075D
:102710003F043F0C6FF04003F7603360002383F306
:102720001188D5F85C28D36863B31069BDE8F0411F
:102730001847230713D014F0080F0CBF0021802185
:10274000E00748BF41F02001A20748BF41F0400127
:10275000630748BF41F48071404600F0EFFBA006DC
:10276000736805D595F8581828461940FEF7CEFD30
:102770003468A4B29FE77060B9E71021281D00F00B
:10278000DDFBC3E7BDE8F08108B50348FFF776FF3E
:10279000BDE8084000F008BCE810002008B5034878
:1027A000FFF76CFFBDE8084000F0FEBB48190020B1
:1027B00008B50348FFF762FFBDE8084000F0F4BB2E
:1027C000A821002010B50E4C0E4A20460021FEF72D
:1027D0006DFD0D4BC4F854380C4C0D4A20460021B9
:1027E000FEF764FD0B4BC4F854380B4C0B4A002128
:1027F0002046FEF75BFD0A4BC4F8543810BD00BFFD
:10280000E81000204D260008004400404819002030
:102810005D26000800480040A82100206D26000821
:102820000078004038B52D4D037A002918BF0D46B9
:10283000012B0446C0F85C580BD1294B984234D187
:10284000284A136C43F4003313640B21262000F054
:1028500027FFD4F85438244A2968934203D002F55C
:102860008062934237D1214AB2FBF1F29A60EA8842
:1028700042F0400292B21A612A8942F0010292B2F9
:102880005A61AA8842F4045141F02C01D96002F443
:10289000A05200211960B2F5806F19685B680CBF07
:1028A0007F23FF2384F8583838BD114B984207D155
:1028B0000C4A136C43F4802313640B212720C6E7D2
:1028C0000C4B9842C5D1074A136C43F08043136404
:1028D0000B215220BBE7084AC6E700BF9C3A00081C
:1028E000E8100020003802400010014000BD010542
:1028F00048190020A821002080DE800200207047B7
:10290000FEE70000704700004FF0FF307047000006
:1029100000F00ABF08B500F075FB00F077FABDE8DB
:10292000084000F0FDB8000070470000022906D002
:10293000032906D00129064818BF00207047054822
:102940007047032A9ABF044800EBC200002070477A
:10295000A03C0008543C00080808002070B504465C
:1029600008460D46FEF78EF9C6B2204601340378BC
:102970000BB9184670BD32462946FEF76BF90028A0
:10298000F3D1012070BD00002DE9F04F81469BB0CE
:1029900008460C461646FEF775F93C49C5B2204676
:1029A000FFF7DCFF08B10235EDB239492046FFF7E9
:1029B000D5FF08B11035EDB2632D01AF0CD8DFF8AB
:1029C000DCA0DFF8DCB03D4694F80080B8F1000FE1
:1029D0001CD185F8008003E02146384600F078FFDE
:1029E0003846FEF74FF9C0B2431C5B0089E8480047
:1029F000337003237370002302361946DAB2904213
:102A000006F102063AD81BB0BDE8F08FB8F1250FE9
:102A10002FD107221D492046FEF71CF958B9DBF8D3
:102A200000202A60DBF804206A609BF808202A72E4
:102A300007340935C8E7082215492046FEF70AF988
:102A4000B8B91448AA1C10F8011F134B4FEA111E05
:102A500001F00F011EF80AE011F80A1002F802EC6A
:102A6000984202F8011C02F10202ECD11835083438
:102A7000AAE785F8008001340135A5E7FA5C06F87D
:102A8000022C06F8011C0133B8E700BFFC3B00082C
:102A9000043C00080F7AFF1F1B7AFF1F173C000839
:102AA0000D3C000808B5202383F311880348FEF786
:102AB0005DFD002383F3118808BD00BF082A0020B4
:102AC00010B50446052916D8DFE801F016150316DF
:102AD000161D202383F311880E4A0121FEF7FCFD09
:102AE00020460D4A0221FEF7F7FD0C48FEF704FDD3
:102AF000002383F3118810BD202383F31188074836
:102B0000FEF7D6FCF4E7202383F311880348FEF791
:102B1000E7FCEDE7AC3B0008D03B0008082A0020AA
:102B200038B50C4D0C4C0D492A4604F10800FFF74E
:102B30002BFF05F1CA0204F110000949FFF724FF39
:102B400005F5CA7204F118000649BDE83840FFF7E0
:102B50001BBF00BFC82E002008080020283C00082A
:102B6000353C0008043C0008BFF34F8F024AD3688D
:102B7000DB03FCD4704700BF003C024008B5094BA2
:102B80001B7873B9FFF7F0FF074B1A69002ABFBF24
:102B9000064A5A6002F188325A601A6822F480624A
:102BA0001A6008BD26310020003C02402301674521
:102BB00008B50B4B1B7893B9FFF7D6FF094B1A6981
:102BC00042F000421A611A6842F480521A601A6890
:102BD00022F480521A601A6842F480621A6008BDBA
:102BE00026310020003C0240172870B513D80B4A4C
:102BF0000B4C137863B90B4E4FF0006144F823106F
:102C000056F823500133182B2944F7D101231370B0
:102C100054F8200070BD002070BD00BF8831002036
:102C200028310020C03C0008014B53F820007047B9
:102C3000C03C000818207047172810B5044601D979
:102C4000002010BDFFF7D0FF064B53F82430184486
:102C5000C21A0BB9012010BD12680132F0D1043B39
:102C6000F6E700BFC03C0008172810B522D8FFF7D0
:102C70007BFFFFF783FF1049F323CB60FFF774FF5F
:102C80000C23B0FBF3F203FB1204D30143EAC403A9
:102C9000DBB243F4007343F002030B610B6943F4AE
:102CA00080330B61FFF760FFFFF782FFBDE8104044
:102CB000FFF7C2BF002010BD003C02402DE9F047E5
:102CC000D40715464DD41318B3F1026F49D2324BD5
:102CD0001B68DA0745D5314CFFF750FFF323E3605B
:102CE000FFF742FF2F46401A40F20129032F884682
:102CF00001EB000618D8294C40F201197B1A434415
:102D0000012B01EB000623692FD823F00103236177
:102D1000FFF74EFF2846BDE8F087366851F8043CBF
:102D2000B34218D1043FE1E7B307E4D1236923F4A8
:102D300040732361236943EA090323610431D8F80E
:102D400000303360BFF34F8FFFF70EFFE368002BB7
:102D5000E3D0F323E360236923F001032361FFF74A
:102D600027FF4FF0FF30BDE8F08723F44073236165
:102D7000236943EA090323618A4631F8023B338021
:102D8000BFF34F8FFFF7F0FE3688BAF80030B6B2C7
:102D9000B342B3D0DFE700BF00380240003C02403E
:102DA000084908B50B7828B153B9FFF7E7FE0123AE
:102DB0000B7008BD23B1BDE808400870FFF7F8BEEE
:102DC00008BD00BF26310020014B186D704700BFC1
:102DD00000280040094B1A6F120407D41A6F42F4FE
:102DE00000721A671A6F42F400421A67044A1368A5
:102DF00043F480731360034B18657047003802403A
:102E00000070004000280040FEE7000010B5184C9C
:102E1000FEF7D0F8FEF74AF800F0A4F88022154932
:102E20002046FEF77FF9012344F8180C0374124B77
:102E3000124AD96821F4E0610904090C0A431049D7
:102E4000DA60CA6842F08072CA600E490A6842F0CD
:102E500001020A601022DA77202283F82220002360
:102E600083F3118862B60848BDE81040FEF788B9C0
:102E7000DC0D0020203D000800ED00E00003FA0515
:102E8000F0ED00E0001000E0283D00082DE9F843D7
:102E9000194C1A4B6769586A002504F114082E462C
:102EA000226ABB68811A8B420CD96169414521D0E5
:102EB00013441B1A022B2CBFC0180230BDE8F84384
:102EC000FEF7E2BB134423623B68D7F80C90C3F8CB
:102ED000048043456361FD6001D1FEF7CFFB86F3BB
:102EE00011883869C847202383F31188034B676929
:102EF000586AD5E7BDE8F883B40D0020000C004007
:102F0000034B59685A68521A9042FBD8704700BF69
:102F1000001000E083691943037C81610A2B03D10F
:102F20004369194205D170470B2B06D143698B4386
:102F300003D100234361FEF745B8704770B50468BC
:102F400005460E46AC4200D170BDE3683343E360F2
:102F500016B12269134203D0A1686068FFF7DAFF57
:102F60002468EFE7034B044A1A60044B044A1A60D2
:102F7000704700BF8C33002090330020883300203E
:102F80000000032080B5074A536823F0010300AF17
:102F90005360EFF30983683383F30988002383F3D5
:102FA000118880BD30EF00E098B5202300AF83F397
:102FB0001188104B5B6813F4006318D0F1EE103ADF
:102FC000EFF309844FF0807344F84C3C0A4BDB6804
:102FD00044F8083CA4F1680383F30988FEF778F805
:102FE00018B1064B44F8503C98BD054BFAE783F303
:102FF000118898BD00ED00E030EF00E021030008EB
:103000002403000808B500F061FB074800F012FC3B
:10301000FEF74AF9FEF73EFBFEF702FAFFF784FCE3
:10302000BDE80840FEF71EBBB03A000830B5039C6F
:103030000172043304FB0325C361049B0363002175
:10304000059B00604060C16042610261856104626D
:1030500042628162C162436330BD00000022416A66
:1030600041610161C2608262C2626FF00101FEF7DC
:10307000E5B8000003694269934203D1C2680AB10E
:1030800000207047181D704703691960C26801323B
:10309000C260C269134482690361934224BF436AD8
:1030A00003610021FEF7BEB838B504460D46E3685B
:1030B0003BB16269131D1268A3621344E3620020EE
:1030C00038BD237A33B929462046FEF79BF80028FD
:1030D000EDDA38BD6FF00100FBE70000C368C2699C
:1030E000013BC3604369134482694361934224BF37
:1030F000436A436100238362036B03B1184770473F
:1031000070B52023044683F31188866A3EB9FFF721
:10311000CBFF054618B186F31188284670BDA36A17
:10312000E26A13F8015BA362934202D32046FFF7E1
:10313000D5FF002383F31188EFE700002DE9F74F57
:103140001F4604460E469146202383F311882A4BDE
:103150005A6A0025BA18009207F1FF3A9846AB4622
:10316000A36AABB91AF1030F06D939462046FFF717
:103170009BFF68B1002305E0D8F82410009A511A8B
:103180008F42F3D283F31188284603B0BDE8F08F55
:10319000A16AE36AA9EB05025B1A934228BF1346B2
:1031A000402B1CD9334601F1400251F8040B43F87F
:1031B000040B9142F9D1A36A40334036A3624035F3
:1031C000A26AE36A9A4202D32046FFF787FF8BF395
:1031D00011884D45D8D2202383F31188C0E71A46C1
:1031E00030460193FDF72CFD019BA26A1A441E4450
:1031F000A2621D44E4E700BF000C004010B5029C31
:103200000172043303FB0421C36100238362C362A0
:10321000039B0363049B00604060C46042610261E1
:10322000816104624262436310BD0000026AC260B1
:10323000426A4261026100228262C2626FF0010151
:10324000FDF7FCBF436902699A4203D1C2680AB123
:1032500000207047184650F8043B0B607047000090
:10326000C368C2690133C36043691344826943611F
:10327000934224BF436A43610021FDF7D3BF00009E
:1032800038B504460D46E3683BB123691A1DA262B6
:10329000E2691344E362002038BD237A33B929463A
:1032A0002046FDF7AFFF0028EDDA38BD6FF00100D2
:1032B000FBE7000003691960C268013AC260C26995
:1032C000134482690361934224BF436A036100236C
:1032D0008362036B03B118477047000070B5202369
:1032E00004460E4683F31188856A35B91146FFF707
:1032F000C7FF10B185F3118870BDA36A1E70A36A61
:10330000E26A01339342A36204D3E169204604399F
:10331000FFF7D0FF002080F3118870BD2DE9F74F33
:103320001F4604460D469146202383F311882A4BFD
:103330005A6A0026BA18009207F1FF3A9846B34637
:10334000A36AABB91AF1030F06D939462046FFF735
:1033500097FF68B1002305E0D8F82410009A511AAD
:103360008F42F3D283F31188304603B0BDE8F08F6B
:10337000A06AE36AA9EB06021B1A934228BF134610
:10338000402B1CD905F1400355F8042B40F8042BC1
:103390009D42F9D1A36A4033A3624036A26AE36A30
:1033A0009A4204D3E16920460439FFF783FF8BF387
:1033B00011884E45D8D2202383F31188C0E71A46DE
:1033C00029460193FDF73CFC019BA26A1A441D4467
:1033D000A2621E44E2E700BF000C0040026943699C
:1033E0009A4203D1C3681BB9184670470023FBE714
:1033F000836A002BF8D0043B9B1AF5D01360C36896
:10340000013BC360C3691A44836902619A4224BFC5
:10341000436A0361002383620123E5E710B50A4490
:103420000024C361029B006040608460C1608161D0
:1034300041610261036210BD08B58269436993422C
:1034400001D1826882B98268013282605A1C42616D
:103450001970426903699A4201D3C368436100212C
:10346000FDF7E0FE002008BD4FF0FF3008BD000072
:1034700070B5202304460E4683F31188A568A5B1D4
:10348000A368A269013BA360531CA361157822695C
:10349000934224BFE368A361E3690BB120469847D8
:1034A000002383F31188284670BD31462046FDF77E
:1034B000A9FE0028E2DA85F3118870BD2DE9F04FEE
:1034C0001E4685B0044688469146D0F81CA02023AD
:1034D00083F31188214F7A6A0293B2180025019272
:1034E000AB46A3681BB3A368013BA360A369591C47
:1034F000A1611B7888F800302369A169994224BF33
:10350000E368A36108F10102BAF1000F03D003924E
:103510002046D047039A8BF31188B9F1010905F1D0
:10352000010516D0029B83F311889046D9E7721EDD
:10353000033207D931462046FDF764FE0028D0D07B
:10354000002304E0796A019A511A8E42F3D283F380
:103550001188284605B0BDE8F08F00BF000C004080
:10356000C16081614161C3611144009B00604060A2
:103570008260016103627047F8B504460E46174643
:10358000202383F31188A568A5B1A368013BA3603C
:1035900063695A1C62611E70236962699A4224BF82
:1035A000E3686361E3690BB120469847002080F32C
:1035B0001188F8BD39462046FDF724FE0028E2DADE
:1035C00085F31188F8BD0000836942699A4210B5FD
:1035D00001D182687AB98268013282605A1C8261A4
:1035E0001C7803699A4201D3C36883610021FDF707
:1035F00019FE204610BD4FF0FF3010BD2DE9F04FF1
:103600001E4685B0044688469146D0F81CA020236B
:1036100083F31188214F7A6A0293B2180025019230
:10362000AB46A3681BB3A368013BA36063695A1C44
:10363000626198F80010197023696169994224BF8A
:10364000E368636108F10102BAF1000F03D003924D
:103650002046D047039A8BF31188B9F1010905F18F
:10366000010516D0029B83F311889046D9E7721E9C
:10367000033207D931462046FDF7C4FD0028D0D0DB
:10368000002304E0796A019A511A8E42F3D283F33F
:103690001188284605B0BDE8F08F00BF000C00403F
:1036A00000F1604300F01F02400903F56143090186
:1036B0008000C9B200F1604083F8001300F561405A
:1036C00001239340C0F8803103607047144B002100
:1036D0001A694FF0FF321A61196158695A615961CC
:1036E000186A60F0805018621962586A5A6259620A
:1036F0001A6C42F080521A640A4A106840F48070D2
:103700001060186F00F44070B0F5007F1EBF4FF4DA
:10371000803018671967536823F40073536070474B
:103720000038024000700040314B4FF080521A6464
:10373000304A4FF4404111601A6842F001021A60A9
:103740001A689207FCD59A6822F003029A609A6878
:103750009A60274B19469A6812F00C02FBD1186840
:1037600000F0F90018609A601A6842F480321A601A
:103770000B689B03FCD54B6F43F001034B671C4B5D
:103780005A6F9007FCD51C4A5A601A6842F0807242
:103790001A60184A53685904FCD5154B1A689201EF
:1037A000FCD5164A9A60164B1A68164B9A42164B6D
:1037B0001AD1164A1168164A914215D140F20512E3
:1037C0001A600B4B9A6842F002029A609A6802F003
:1037D0000C02082AFAD15A6C42F480425A645A6E9A
:1037E00042F480425A66704740F20572E8E700BF33
:1037F0000038024000700040185440070094883898
:10380000002004E011640020003C024000ED00E0D4
:1038100041C20F414B6843608B688360CB68C360D3
:103820000B6943614B6903628B6943620B680360F8
:10383000704700001C4B0246186B10B540F2FF1495
:1038400020431863196D1948214319651146FFF784
:10385000E1FF174802F11C01FFF7DCFF154802F1F8
:103860003801FFF7D7FF144802F15401FFF7D2FFE8
:10387000124802F17001FFF7CDFF114802F18C01EF
:10388000FFF7C8FF0F4802F1A801FFF7C3FF0E487A
:1038900002F1C401FFF7BEFF0C4802F1E001BDE8F0
:1038A0001040FFF7B7BF00BF0038024000000240E1
:1038B0000004024000080240000C024000100240D8
:1038C0000014024000180240001C02400020024088
:1038D00080EA0102844612F0030F4FD111F0030F6A
:1038E00032D14DF8044D11F0040F51F8043B0BD0C8
:1038F000A3F101329A4312F0803F04BF4CF8043B1D
:1039000051F8043B16D100BF51F8044BA3F101322A
:103910009A4312F0803FA4F101320BD14CF8043BE2
:10392000A24312F0803F04BF51F8043B4CF8044B13
:10393000EAD023460CF8013B13F0FF0F4FEA332384
:10394000F8D15DF8044B704711F0010F06D011F863
:10395000012B0CF8012B002A08BF704711F0020F51
:10396000BFD031F8022B12F0FF0F16BF2CF8022B3C
:103970008CF8002012F47F4FB3D1704711F8012B5F
:103980000CF8012B002AF9D1704700BF1210121356
:103990001211000053544D3332463F3F3F000000A8
:1039A000012033000010410101105A010310590198
:1039B0000710310100000000943900083F000000AA
:1039C00013040000F43900083F000000190400004F
:1039D000FE3900083F00000021040000083A0008FA
:1039E0003F000000082A0020E810002048190020AD
:1039F000A821002053544D333246343078005354BC
:103A00004D3332463432780053544D3332463434D9
:103A10003658580075120008611200089D120008FF
:103A20008912000895120008811200086D12000822
:103A3000591200089D13000889130008C5130008D7
:103A4000B1130008BD130008A9130008951300085E
:103A500081130008000000000100000000000000C9
:103A600000000000D9170008B51A0008511B000813
:103A700040004000D0100020D010002001000000C5
:103A8000E010002080000000400100000300000062
:103A90007573625F70756D70000000000096000025
:103AA0000000000000000000000000000000000016
:103AB0000000802A00020000AAAAAAAA00000000B2
:103AC000FFFF00000000000000A00A00000000004E
:103AD00000000000AAAAAAAA00000000FFFF000040
:103AE00000000000000000000000000000000000D6
:103AF000AAAAAAAA00000000FFFF00000000000020
:103B00000000000080298A0100000000AAAAAAAAD9
:103B100080148500FFFF00000070700777700000C0
:103B20000080020100000000AAAAAAAA0040010029
:103B3000FFFF0000000000800800000000000000FF
:103B400000000000AAAAAAAA00000000FFFF0000CF
:103B50000000000000000000000000000000000065
:103B6000AAAAAAAA00000000FFFF000000000000AF
:103B70000000000000000000000000000A0000003B
:103B80000000000003000000000000000000000032
:103B90000000000000000000000000000000000025
:103BA0000000000000000000000000000200000013
:103BB00000000000B9150008211600084000400070
:103BC000982E0020A82E0020020000000000000017
:103BD0000300000000000000611600080000000063
:103BE00010000000B82E00200000000001000000BE
:103BF00000000000F80D00200101020025424F41A5
:103C0000524425002553455249414C2500437562D5
:103C100065426C61636B003031323334353637388E
:103C200039414243444546004865782F50726F66DB
:103C300069434E430043756265426C61636B2D427C
:103C40004C000000C12A00082D2900082515000895
:103C5000A52A0008430000005C3C0008090243005C
:103C6000020100C032090400000102020100052423
:103C700000100105240100010424020205240600AD
:103C800001070582030800FF09040100020A000081
:103C90000007050102400000070581024000000006
:103CA00012000000A83C00081201100102000040B0
:103CB000AE2D0110000201020301000004030904FB
:103CC00000400000004000000040000000400000F4
:103CD00000000100000002000000020000000200DD
:103CE00000000200000002000000020000000200CC
:103CF00000400000004000000040000000400000C4
:103D000000000100000002000000020000000200AC
:103D1000000002000000020000000200000002009B
:103D20006D61696E00000000403D00089031002088
:103D30008833002001000000092E00080000000068
:103D400069646C6500000000FF0096000000000838
:103D500004000000BC3C000800000000000000005F
:103D60000000000000000000000000000000000053
:00000001FF
